:10000000B4011029B600A52084133230A6000030B8
:10001000A700F020A00AA50AA201A3010008360546
:10002000A600640000083605A70026062705360648
:100030000319A20A0319A30A2708A600A403031997
:10004000A5030319A00B112822080B290408A700F7
:100050008611051205128316861105120512F0305D
:10006000850583122708B41853283A30A100983028
:10007000B6203330A60068201330A1008830B620A7
:1000800068206430B52068206430B5202230A60096
:100090006820283052200C30522006305220B414F0
:1000A000270853283414A600341C61280512033C89
:1000B000031C662866200730A100D030B620031448
:1000C00008003414FE3C03190B290516A60E341C37
:1000D00034108615F030850526080F398504861101
:1000E000A60E341868283230B52003140800B51362
:1000F00029080319B5170530A8002730A3001030D0
:100100008D200330A300E8308D20A30164308D20C2
:10011000A3010A308D2024089428A2002508A100FC
:100120002408A000D4202008A000A8030319B513B8
:10013000290803199E282802031808002008031D17
:10014000B513B51B0800303E0629841780040B291F
:10015000A301A200FF30A207031CA307031C0B2965
:100160000330A100DF30B620AA28A101E83EA0009C
:10017000A109FC30031CBF28A0070318BC28A00756
:100180006400A10FBC282018C528A01CC9280000A5
:10019000C9280800013EA7000A30A200A301D4200C
:1001A000A70BCF2824080800A501A4011030A60041
:1001B000210DA40DA50D2208A4022308031C230F62
:1001C000A5020318EA282208A40723080318230F0E
:1001D000A5070310A00DA10DA60BD82820080B29F8
:1001E0001030A800A101A001A70CA60C031CFE283A
:1001F0002208A00723080318230FA107A10CA00CB5
:10020000A50CA40CA80BF42824080B2984003108A1
:100210008A003008820083130313831264000800ED
:10022000831603308600831207309F00BC01BD0196
:100230000330A300E830A920FE302720013027201A
:10024000FE30272001302720FE3027208030272055
:10025000203027204D302720693027206B30272081
:100260006530272020302720463027207230272075
:1002700065302720653027206D302720613027200A
:100280006E3027202030272020302720FE302720E6
:10029000C030272020302720203027203030272052
:1002A000383027202D3027203030272033302720AA
:1002B0002D302720303027203730272020302720AE
:1002C0002030272020302720203027200330A30093
:1002D000E830A920FE302720013027206430A820F4
:1002E000DC30A2000530A300063084000430022078
:1002F000BA002308BB003A08A6003B08A700143048
:10030000A200A301F020BA002508BB006400061C6F
:100310008D293A08BC003B08BD00FE302720803004
:10032000272052302720503027204D3027202030E2
:1003300027203D30272020302720A9013A08A0009F
:100340003B08A1000330CA20B200B3013208A40068
:100350003308A5002630B000B1017720A9013A0882
:10036000A0003B08A1000230CA20B200B30132084D
:10037000A4003308A5002630B000B1017720A90100
:100380003A08A0003B08A1000130CA20B200B30126
:100390003208A4003308A5002630B000B101772050
:1003A000A9013A08A0003B08A1000030CA20B20011
:1003B000B3013208A4003308A5002630B000B10113
:1003C0007720FE302720C03027204D3027204530B1
:1003D00027204D302720203027203D302720203077
:1003E0002720A9013C08A0003D08A1000330CA2035
:1003F000B200B3013208A4003308A5002630B000D3
:10040000B1017720A9013C08A0003D08A1000230FD
:10041000CA20B200B3013208A4003308A500263078
:10042000B000B1017720A9013C08A0003D08A1005F
:100430000130CA20B200B3013208A4003308A5007D
:100440002630B000B1017720A9013C08A0003D088A
:10045000A1000030CA20B200B3013208A400330862
:10046000A5002630B000B1017720FE3027200230F1
:080470002720702963003A2ADD
:02400E00543F1D
:00000001FF
